:1000000000308A008B280000831A0A28A400030EFF
:10001000A5000F288312A400030EA500A5140A084A
:10002000AB008A018313A40E0408A6002008A700D1
:100030002108A8002208A9002308AA0083128C30F6
:100040008400001C25280C1838282608840027085E
:10005000A0002808A1002908A2002A08A3002B0854
:100060008A00250E83008312240EA518831609002A
:10007000FF30AC020318AD020030031C0130AE02A9
:100080000030031C0130AF02AF08031D5B282E08AF
:10009000003C031C5B284030AC074B3003184C304D
:1000A000AD074C3003184D30AE0700300318013057
:1000B000AF070130B4000C108A11252839308400B4
:1000C0000008031970280630A100A001A00B6628C3
:1000D000A10B65287B30A000A00B6C28800B632847
:1000E00008008316051083120514831685108312E9
:1000F0008510370B7D28C8307E286430B80038085A
:10010000B9005E2083160510831205108316851032
:1001100083128514080003081F3983003F30A000B4
:100120002130840083138001840AA00B9328A0014E
:1001300084011F308305AF01AE010330AD00E8300C
:10014000AC000830B000B201B101B301B401073016
:10015000990083160108C7390838810007308312D7
:10016000990083160508850010308312A000A00BAB
:10017000B728000019088C1183160510831205108A
:1001800083168510831285140C30B600FA30B9003E
:100190005E20B60BC628AF014C30AE004B30AD0030
:1001A0004030AC000530900083160C1408308312E8
:1001B000B000B201B101B301B401310883169B0054
:1001C0009C131C141A088312B500C0308B04B508A8
:1001D00003191D29340B1C29B40133083A3C031CB4
:1001E0001B293308123C031CF828B7017120192978
:1001F000B0033508A0003008A1000319032903103B
:10020000A00CA10BFF28003020180130B600B70069
:100210007120B008031D19290830B000B10A031974
:10022000B20A310883169B009C131C141A0883120F
:10023000B500B30A1C29B301E7280B138B138B1BE2
:100240001E2983160510831205108316851083124C
:1002500085145030B600FA30B9005E20B60B2B2959
:060260008316D62863009E
:104200005A00640035002400D2007A0024003500F2
:104210002400D2004600240035002400D2006600AD
:10422000640035002400D200410024003500240041
:10423000D2006100240035002400D20011002400C7
:1042400035002400D2007100640035002400D20043
:1042500049002400B5002400D20069006400350044
:104260002400D2005900640035002400D2007900F7
:10427000240035002400D30045002400350024002C
:10428000D2006500640035002400D2004300240001
:0842900035002400D2000000FB
:02400E00C23FAF
:00000001FF
